:100000009D28AB004230A3000F30A40066200319E6
:100010001210031D1214FC3E031C921003189214BC
:100020004030A3004230A4000F30A700A8011218EE
:1000300037209218372068202303831692008312FA
:100040002308A5002408A6002008A900AA00200F64
:10005000AA018220280895000C309700A71B97164C
:10006000271B17168316061183121215982838209D
:100070000310A70CA40CA30C080083178001840AAA
:10008000FF3E031D3E289828A601A500FF30A507C6
:10009000031CA607031C98280330A400DF3052205D
:1000A0004628A401E83EA300A409FC30031C5B28F9
:1000B000A30703185828A3070000A40F58282318E3
:1000C0006128A31C6528000065280800A801A70175
:1000D0001030A900240DA70DA80D2508A702260899
:1000E000031C260FA80203187C282508A70726084A
:1000F0000318260FA8070310A30DA40DA90B6A2847
:10010000230898281030AC00A401A301AA0CA90C64
:10011000031C90282508A30726080318260FA40708
:10012000A40CA30CA80CA70CAC0B862827089828B5
:100130008313831203130000080007309F00831607
:10014000811320308400603083123E20A030840070
:1001500050303E202030840030303D208501860123
:10016000F03083168500FF3086008312D32AA00169
:100170000930A600C430A500013001208316861581
:10018000831205150330B600E830B5008510B801BC
:100190000130B7003808031DE0285130370203183A
:1001A000E02883160510831205143608A4003508CC
:1001B0005220051014304420B70A0319B80FCA287A
:1001C000851485113010B010B201B101033006055D
:1001D000A201A1002108033A2204031DFD28B10A4F
:1001E0000319B20A32082E3AE03003193106031D12
:1001F000FA28D32A0A304420E62814304420033059
:100200000605A201A1002208031D112903302102C5
:100210000318112906180D29301486181029B01456
:10022000FF28030130180130AF000301B01801307E
:100230002F0503191C29462A301C20290A30B90031
:10024000B01C2429C830B900851585100430360249
:10025000031C3029031D412975303502031841293B
:1002600083160510831205143608A40035085220A1
:100270000510143044200230B507031C2629B60FA0
:1002800026290130BA003A083902031CD629013068
:100290003A02031D72290A303902031D6E29B80182
:1002A0000130B7003808031D6D290B3037020318E1
:1002B0006D290130A600F430452006186029E22A95
:1002C00085110130A600F4304520851506186929EE
:1002D000E22AB70A0319B80F522972290730A6007B
:1002E000D030452005303602031C7C29031D90299F
:1002F0001530350203189029831605108312051452
:100300003608A40035085220051014304420061881
:100310008A29E22A0530B507031C7229B60F722913
:10032000C7303A02031DA829831686117F30831235
:10033000A0000330A600E830A50001300120B43051
:100340004420A001A601A5010130012083168615D5
:1003500083120430A600B03045200530B502031CDE
:10036000B60304303602031CD429031DBB29103008
:100370003502031CD4298316051083120514360890
:10038000A400350852200510143044200618C9294D
:10039000E22A0530B50200300318D129013E0318C6
:1003A000D429B6020318B129BA0F43290430B60084
:1003B0001030B50003303602031CFA29031DE4296E
:1003C000E8303502031CFA29831605108312051440
:1003D0003608A4003508522005101430442002309D
:1003E000B50200300318F729013E0318FA29B602B6
:1003F0000318DA29B8010130B7003808031D132AA1
:100400000B3037020318132A8316051083120514C4
:100410003608A40035085220051014304420B70ACD
:100420000319B80FFD298514831686110130831234
:10043000BD0004303D020318422AA530BC003C0830
:10044000A0000930A600C430A500013001203C09FD
:10045000A1000310210CAD00AE012E08AA002D084A
:10046000A900A6013C30A5008220A3002808A40012
:10047000230852200130BC0203181F2AC830442030
:10048000BD0F192A831686158312B7288515831682
:10049000861101308312BD0002303D020318A12AEB
:1004A000B401FA30B30007303402031C5D2A031D87
:1004B000762AD13033020318762A7F30A000340820
:1004C000A6003308A5000130012001300618030101
:1004D000AF000130861803012F040319702AB728D2
:1004E0001930B307031C532AB40F532A0730B40042
:1004F000D030B3003408031D812AFA303302031CC4
:100500009F2A7F30A0003408A6003308A5000130E0
:100510000120013006180301AF00013086180301E5
:100520002F040319942AB7280730B30200300318A8
:100530009C2A013E03189F2AB40203187A2ABD0F91
:100540004C2A8316861501308312BD00C9303D0246
:100550000318B92A05304420013006180301AF0002
:100560000130861803012F040319B72AB728BD0FDD
:10057000A62A8510B8010130B7003808031DD32A18
:10058000513037020318D32A83160510831205143D
:100590000730A400D0305220051014304420B70A90
:1005A0000319B80FBD2A8514051185118316861508
:1005B00001308312A6002C3045200B168B106300EF
:1005C0000B12B72803303602031C022B031DEC2A42
:1005D000E8303502031C022B831605108312051424
:1005E0003608A4003508522005101430442002308B
:1005F000B50200300318FF2A013E0318022BB60291
:060600000318E22AB728EE
:02400E00303F41
:00000001FF
